:1000000000308A00BC2800000A108A100A118207FA
:1000100050346534723469346F346434613420345C
:10002000253435344C3475342034753473342E34DF
:100030000A340D340034F701F801F901FA01BF0167
:10004000C001C101C2013E083D043C043B04031948
:1000500059282030C3000310B70DB80DB90DBA0DE3
:10006000BF0DC00DC10DC20D3E084202031D422846
:100070003D084102031D42283C084002031D42285E
:100080003B083F02031C53283B08BF023C08031CEB
:100090003C0FC0023D08031C3D0FC1023E08031C7B
:1000A0003E0FC2020314F70DF80DF90DFA0DC30B44
:1000B0002B283F308400831300340408AF003B300A
:1000C000B6009A30B500CA30B400B3010A30B100AE
:1000D0002E08BA002D08B9002C08B8002B08B7006C
:1000E0003608BE003508BD003408BC003308BB002C
:1000F0001B200008AB00840A0008AC00840A00083A
:10010000AD00840A0008AE00F708031D9A283108E4
:10011000013A03199A282F0803199B280F39310235
:10012000031994280318A128AF1BA1282F1B9B2873
:1001300020309C28AF013030F70777080C1E9E282E
:1001400099003608BA003508B9003408B8003308F9
:10015000B700BE01BD01BC010A30BB001B207A08FC
:10016000B6007908B5007808B4007708B300B10B81
:1001700068288A110A128229840183131F3083059B
:10018000193083169900A630980090308312980099
:1001900083161F149F141F159F1107309C00FF30FA
:1001A0008312A00083161F149F141F159F11831222
:1001B0001F109412A01220088316870083122016A5
:1001C0002008831687008312A01120088316870059
:1001D0000130831294000030831694000108C7395F
:1001E000083881008530831290000030F8009200BA
:1001F00000308316920007309C000508640002302E
:10020000F700F70B012904291C0883120D1383162C
:100210009D018601FF3083128600A701A601A5017A
:10022000A401A3012308093C031C542983160516C5
:100230008312051A1629831605168312051E1B291B
:10024000831605168312051E2D298F018E01831634
:1002500005168312051A27292029831605168312ED
:10026000051A3829831605168312051E32292D29F1
:100270000F08FA000E08F7000F087A02031D38294C
:100280007708A1007A08A2002108A4072208031811
:10029000220FA507003003180130A607003003180D
:1002A0000130A707A30A12292708BA002608B900B7
:1002B0002508B8002408B700BE01BD01BC01230811
:1002C000BB001B207A08A7007908A6007808A500C3
:1002D0007708A400AA012A080420AA0AF7007708D0
:1002E0000C1E7029990008302A02031D6B29053065
:1002F00084002708AE002608AD002508AC002408BD
:10030000AB005D280C30AB002B080420AB0AF700D3
:1003100077080C1E8929990012302B02031D8429AD
:10032000DA302402F7002508F8000B30031C0C30EB
:10033000F8022608F9000030031C0130F9022708F2
:10034000FA000030031C0130FA027808A90077088F
:10035000A800A91FBA292908FF3C031CBA29031DBC
:10036000B5292808CA3C031CBA2983168601BF3068
:1003700083128600A91FC7292908FE3C0318D82923
:10038000FF3A031DC7292808CB3C0318D829A91F09
:10039000D8292908FF3C031CD829031DD329280884
:1003A000DC3C031CD82983168601DF3083128600CB
:1003B000A91FE5292908FE3C0318F629FF3A031D69
:1003C000E5292808DD3C0318F629A91FF629290884
:1003D000FF3C031CF629031DF1292808EE3C031CF1
:1003E000F62983168601EF3083128600A91F032A9F
:1003F0002908FE3C0318112AFF3A031D032A280886
:10040000EF3C0318112AA91B0C2AA908031D112A65
:100410002808103C031C112A83168601F73083122A
:100420008600A91B282AA908031D1A2A2808113C9E
:100430000318282AA91B232AA908031D282A2808EB
:10044000223C031C282A83168601FB308312860077
:10045000A91B3F2AA908031D312A2808233C031899
:100460003F2AA91B3A2AA908031D3F2A2808333C22
:10047000031C3F2A83168601FD3083128600A91BC8
:100480004D2AA908031D482A2808343C03184D2A80
:0E04900083168601FE30831286000D2963005C
:02400E00393F38
:00000001FF
